:100000000C9402030C9446030C9446030C94460390
:100010000C9446030C9446030C9446030C9446033C
:100020000C9446030C9446030C941C0E0C94EE0E98
:100030000C9446030C9446030C9446030C9446031C
:100040000C9446030C94F8220C9446030C9446033B
:100050000C9446030C948B1C0C9446030C9446039E
:100060000C9446030C9446030C9446030C944603EC
:100070000C9446030C9446030C9446030C944603DC
:100080000C9446030C9446030C9446030C944603CC
:100090000C9446030C9446030C9446030C944603BC
:1000A0000C9446030C9446030C9446035B0F7D0F9F
:1000B0006B107D0F6B10C20FE50F6B103A104D10D7
:1000C0001C131C134B134B138113A113D214D21402
:1000D000AC13D2145C145C14C314D214D214CC1418
:1000E0006914691469146914691469146914691428
:1000F0006914691469146914691469146914691418
:100100007B1488148F149614A0140147024774328C
:10011000014702477432012102217432012802286A
:10012000000147024774320147024774320120023E
:100130002074320128022800014702477432014727
:1001400002477432011F021F743201280228000185
:100150004702477432014702477432011E021E747F
:10016000320128022800000001C002C003C004C000
:1001700005C0018C028C2E004C002900E1003542A4
:1001800000001E00140004001D0034004D421F003A
:100190001A0015001B00E1042A7120000900160056
:1001A000060050002C7221001300170019004F00A8
:1001B0004A0022000A00070005000000E20050008B
:1001C000025400002E00000001204F0002540000E5
:1001D0002D000000E20023000D000B000E000000C7
:1001E000E60024000F001100100052004B00250013
:1001F0001800080036005100287226001C000C0070
:1002000037002F002B7127003300120038713000A7
:100210004E432D0031003400E500004200002E0066
:100220004C002900E100354200001E0014000400CB
:100230001D0034004D421F001A0016001B00E1048F
:100240002A71200008000700060050002C722100CF
:100250001500090019004F004A00220017000A008B
:1002600005000000E2005000025400002E000000D3
:1002700001204F00025400002D000000E200230086
:100280001C000B0011000000E600240018000D0007
:10029000100052004B0025000C000E0036005100EB
:1002A0002872260012000F0037002F002B71270044
:1002B00013003300387130004E432D0031003400FC
:1002C000E500004200000100010001000100010002
:1002D00000003A001E0220022202010001003B0041
:1002E0001F0221022302010001003C002F0226020E
:1002F0002F00010001003D00300227023000010004
:1003000001003E003102350035020000010001000D
:1003100001000000010000000100010001000000D8
:100320000100000001003F005200510024020000C3
:1003300001004000240021001E00010001004100D6
:10034000250022001F003700010042002600230084
:10035000200027000100430025022E0231002E005C
:100360000100440045000100010001000000000000
:100370000000000000000000000000000620022035
:100380000000000001000000072003200000000022
:100390000100000000000420000000000100000037
:1003A0000000052000000000010000000000000027
:1003B000000000000100000000000000000000003C
:1003C000010000000000000000000000010000002B
:1003D000000000000000000001000000000000001C
:1003E000000000000100000000000000000000000C
:1003F00001000000000000000000000001000000FB
:1004000000000000000000000100000000000000EB
:1004100000000000000016034500720067006F0036
:1004200044006F007800200045005A0000001603C9
:100430004500720067006F0044006F0078002000E4
:1004400045005A0000000403090409026D0004017C
:1004500000A0FA09040000010301010009211101B3
:100460000001223F000705810308000A090401007A
:100470000103010200092111010001224D000705BD
:10048000820308000A090402000103000000092198
:10049000110100012236000705830308000A090440
:1004A00003000103000000092111010001223900AD
:1004B000070584031000011201100100000008ED7F
:1004C000FE071301000102000105010906A1010553
:1004D0000719E029E7150025019508750181020536
:1004E000081901290595057501910295017503917A
:1004F00001050719002977150025019578750181F7
:1005000002C005010980A101850216010026B7007D
:100510001A01002AB700751095018100C0050C0969
:1005200001A1018503160100269C021A01002A9CE4
:1005300002751095018100C005010902A1010901A0
:10054000A100050919012905150025019505750169
:100550008102950175038101050109300931158179
:10056000257F95027508810609381581257F95013B
:1005700075088106050C0A38021581257F950175DD
:10058000088106C0C005010906A101050719E02977
:10059000E71500250195087501810295017508810F
:1005A0000105081901290595057501910295017547
:1005B0000391010507190029FF150025FF95067510
:1005C000088100C0000000000000000000000001E1
:1005D0000204060A0F17202C3A4A5D71879DB3C7A3
:1005E000DAE9F5FCFFFCF5E9DAC7B39D87715D4AEE
:1005F0003A2C20170F0A0604020100000000000038
:100600000000000011241FBECFEFDAE0DEBFCDBF37
:1006100004B603FE24C08091FB019091FC01A091DF
:10062000FD01B091FE018730904BA740B04BB9F46B
:100630001092FB011092FC011092FD011092FE013C
:1006400014BE84B7877F84BF88E10FB6F894809387
:100650006000109260000FBEE0E0FFE3099511E03A
:10066000A0E0B1E0EEE7F9E402C005900D92A433FA
:10067000B107D9F711E0A4E3B1E001C01D92AB3F8F
:10068000B107E1F70E94600B0C94BD240C940000AC
:100690001092B9008AE08093B800089594EA90938C
:1006A000BC009091BC0097FFFCCF9091B900987F5F
:1006B000983021F0903111F081E008958093BB00D3
:1006C00084E88093BC008091BC0087FFFCCF8091C0
:1006D000B900887F883111F0803471F780E0089587
:1006E00084E98093BC008091BC0084FDFCCF089518
:1006F0008093BB0084E88093BC008091BC0087FF9E
:10070000FCCF9091B900987F81E0983209F480E0A5
:10071000089584E88093BC008091BC0087FFFCCFE3
:100720008091BB00089580910101811115C080E482
:100730000E944E038093010181110CC082E10E944E
:10074000780380930101811105C08FEF0E94780327
:10075000809301010E94700384B1807F84B985B1C8
:10076000807F85B98AB1837F8AB98BB1837F8BB94A
:100770003E98469808950E944E05809301010E947C
:10078000930380B38C7080BB81B3836F81BBA5E37F
:10079000B1E0E3E4F1E08EE08E0F11921D928E1332
:1007A000FCCF0C943805BF92CF92DF92EF92FF926C
:1007B0000F931F93CF93DF9380910101882379F0EA
:1007C000809134018F5F80933401811108C00E94B1
:1007D0004E0580930101811102C00E94E00405E3EF
:1007E00011E0C0E0D0E0DD24D39482E0C82EEE24F6
:1007F000E394F12CC730D10500F5809101018111FE
:1008000064C080E40E944E0380930101811112C0F4
:1008100082E10E9478038093010181110BC0C7011E
:100820000C2E01C0880F0A94EAF780950E94780385
:10083000809301010E94700348C0CA30A1F028F4DF
:10084000C83059F0C93061F005C0CC3089F070F083
:10085000CD3089F0209A289810C0219A29980DC08F
:10086000229A2A980AC0239A2B9807C0529A01C04C
:10087000539A5B9802C03E9A469890EA9A95F1F78F
:100880009FB1799902C082E001C080E091709D25FE
:10089000982B7C9902C084E001C080E0892B7D996F
:1008A00002C038E001C030E0832B7E9902C020E115
:1008B00001C020E0822B9FB19095991F9927991F25
:1008C0009295990F907E892B0FC080910101811123
:1008D00049C080E40E944E0380930101882379F18E
:1008E000B12C0E9470038B2DF8019081981719F09C
:1008F0008083C09200010E94930321960F5F1F4FD7
:10090000CE30D10509F076CF80910001882361F1C6
:10091000815080930001882339F08FE99FE001978F
:10092000F1F700C0000020C0A3E4B1E0E5E3F1E08E
:10093000CF01825F91919D938E13FCCF15C083E10F
:100940000E947803809301018111CACF81E40E9443
:100950004E03809301018111C3CF0E948903B82EF9
:10096000B094BFCF80E0C0CF0E94DE0481E0DF9171
:10097000CF911F910F91FF90EF90DF90CF90BF909C
:100980000895E82FF0E0ED5BFE4F80810895089513
:100990000F931F93CF93DF93C3E4D1E010E00C2FAC
:1009A000025F899190E00E94B11B180F0C13F9CFE0
:1009B000812FDF91CF911F910F9108950C94E00545
:1009C00056985E9825982D9826982E9827982F98B7
:1009D0008FEF90E0909389008093880090938B0034
:1009E00080938A0090938D0080938C00259A2D9A95
:1009F0002FEF80E792E0215080409040E1F700C067
:100A00000000269A2E9A2FEF80E792E02150804036
:100A10009040E1F700C00000279A2F9A2FEF80E75F
:100A200092E0215080409040E1F700C000002598FE
:100A30002D982FEF80E792E0215080409040E1F721
:100A400000C0000026982E982FEF80E792E02150FA
:100A500080409040E1F700C0000027982F985698FA
:100A60005E9825982D9826982E9827982F98089567
:100A700089EA8093800089E08093810024982C98F3
:100A80003F988AB18F748AB96E98479A8BB1806B00
:100A90008BB9769A0E94E0040C94DF0580E2809383
:100AA00001018091510181110EC00E94480381E033
:100AB000809351012FEF83ED90E3215080409040CF
:100AC000E1F700C0000080E40E944E038093010122
:100AD00081112EC00E94780380930101811128C0EA
:100AE0000E94780380930101811122C08FE30E944C
:100AF00078038093010181111BC00E94700380E480
:100B00000E944E0380930101811112C08CE00E946B
:100B100078038093010181110BC00E9478038093B8
:100B20000101811105C08FE30E94780380930101C8
:100B30000E947003809101010895FC01623021F14F
:100B400028F4662349F0613071F036C0643041F119
:100B500008F1653059F130C08281882311F085EEAB
:100B60000CC085EE0EC08281882351F085EE0E9474
:100B7000C01185EE0E94881283EE0E94C0111CC035
:100B800083EE0E94881218C08281811115C08FE403
:100B900091E00895828181110FC088E391E008956A
:100BA0008281811109C081E291E0089582818111E1
:100BB00003C08AE091E0089580E090E008950895F0
:100BC0006091BD017091BE018091BF019091C00103
:100BD0000E94BD1B56985E9825982D9826982E98B1
:100BE00027982F98823019F0833021F00895259AA4
:100BF0002D9A0895269A2E9A089581E0089581E00D
:100C000008950C94FF0508950F931F93CF93DF93DE
:100C10008C01FC01C081D181CE010E94361ABE0137
:100C20000E94AD06EC01B8010E940106882309F478
:100C30008DC0F8018281882309F44AC080915D014A
:100C400081111FC0C431F0E5DF0709F051C00E94D7
:100C5000030681E080935D010E94551C90935C0126
:100C600080935B011092540110925601109255012D
:100C7000109258011092570110925A011092590186
:100C800065C080915B0190915C010E94611C883C71
:100C9000910570F480915401E82FF0E0EE0FFF1FF2
:100CA000EB5AFE4FD183C0838F5F809354014EC0B7
:100CB000C43880E5D80721F0C538D04501F13AC0E5
:100CC000F8018281882341F01092520182E01EC017
:100CD000C438E0E5DE0759F580915201811106C064
:100CE00086E20E94C01186E20E94881282E01CC047
:100CF000C438F0E5DF0741F3C538D045D9F4F80131
:100D00008281882331F01092530180E20E94D71231
:100D10001DC080915301811106C087E20E94C0115D
:100D200087E20E94881280E20E94DE120FC0C5385E
:100D3000D04529F381E08093520180935301C8018B
:100D4000DF91CF911F910F910C94FD0580E0DF9111
:100D5000CF911F910F910895089596E0799FF0012A
:100D6000112494E5899FE00DF11D1124E60FF11D7A
:100D7000EE0FFF1FEA58FE4F859194910895880F5A
:100D8000991FFC01EA51F040859194910895880FD4
:100D9000991FFC01EA59FE4F8591949108950F9394
:100DA0001F93CF93DF93EC01811520E3920750F559
:100DB000C11580E2D80708F0C3C0CB3BD10590F441
:100DC000C83AD10508F06AC0C53AD10508F05BC041
:100DD000C430D10508F0D0C1219709F0CAC101E0A3
:100DE00010E00AC2CF3FD10511F008F0C5C1C03FE5
:100DF000D10508F0A2C0CE01805E9109089708F4E1
:100E0000BBC1B7C1C13090E5D90709F4A2C020F534
:100E1000C0318FE4D80770F4C11590E4D90708F009
:100E200094C0C11521E3D20708F0A3C1DD278E01CC
:100E3000106CE2C1C115D04509F09BC10E943D155F
:100E40008FEF94E32CE0815090402040E1F700C008
:100E500000000E94B01CD0C1C11597E5D90758F415
:100E6000C03121E5D20708F01CC1C43180E5D807A4
:100E700008F475C07EC1CE0190578115904108F0ED
:100E800078C1DF7073C1C53AD10509F477C1C63A9C
:100E9000D10509F076C102E810E4AEC1C83AD10527
:100EA00009F472C1C93AD10509F471C1CA3AD10530
:100EB00009F470C1CB3AD10509F46FC1CC3AD10520
:100EC00009F46EC1CD3AD10509F46DC1C03BD1051D
:100ED00009F46CC1CE3AD10509F46BC1CF3AD10502
:100EE00009F46AC1C13BD10509F469C1C23BD1050E
:100EF00009F468C1C33BD10509F467C1C43BD105FE
:100F000009F466C1C53BD10509F465C1C63BD105ED
:100F100009F464C1C73BD10509F463C1C83BD105DD
:100F200009F462C1C93BD10509F461C1CA3BD105CD
:100F300009F460C100E014E45FC18E0110655CC17A
:100F4000CE019F700E94C70658C1DF708E01106AE3
:100F500053C18091DA0181608093DA014DC10E9412
:100F6000551E811102C00E943B1E0E94721E90E01D
:100F70009093FB018093FA01C23080E5D80721F4F9
:100F80008091FA01816086C0C43090E5D90721F4D0
:100F90008091FA0182607EC0C63020E5D20721F43C
:100FA0008091FA01846076C0C83080E5D80719F4D2
:100FB0008091FA0127C0CA3090E5D90721F48091C9
:100FC000FA01806167C0CC3020E5D20721F480911E
:100FD000FA0180625FC0CE3080E5D80721F48091AD
:100FE000FA01806457C0C03190E5D90721F480919F
:100FF000FA0180684FC0C23120E5D20729F4809100
:10100000FA018460886046C0C33080E5D80721F4C7
:101010008091FA018E7F3EC0C53090E5D90721F45A
:101020008091FA018D7F36C0C73020E5D20721F4C8
:101030008091FA018B7F2EC0C93080E5D80719F462
:101040008091FA0126C0CB3090E5D90721F4809138
:10105000FA018F7E1FC0CD3020E5D20721F48091A8
:10106000FA018F7D17C0CF3080E5D80721F4809139
:10107000FA018F7B0FC0C13190E5D90721F480912F
:10108000FA018F7707C0C331D04531F48091FA015E
:101090008B7F877F8093FA018091FA010E94761EF0
:1010A000ABC08D2F99278F70992781309105D9F486
:1010B0009E012370332702C0880F991F2A95E2F7FB
:1010C0009C688E0144E0000F111F4A95E1F700274C
:1010D0001370802B912B53E0CC0FDD1F5A95E1F755
:1010E000C076DD272FC08230910531F4DC2FCC276C
:1010F0008E01016F106A80C08330910569F4CE01C2
:101100008370992701E010E002C0000F111F8A953B
:10111000E2F7C8019C680FC084309105B9F4CE0194
:101120008370992701E010E002C0000F111F8A951B
:10113000E2F7C8019A6823E0CC0FDD1F2A95E1F79A
:10114000C07ED7708C010C2B1D2B56C085309105AD
:1011500031F4DC2FCC278E01046F106A4DC0069746
:1011600009F04AC0CF71DD27DC2FCC278E01106239
:1011700043C000E010E040C08E013EC001E810E432
:101180003BC003E810E438C002EE14E435C009EEB9
:1011900014E432C00AEE14E42FC005EB14E42CC0B2
:1011A00006EB14E429C007EB14E426C00CEC14E4AD
:1011B00023C00DEC14E420C003E815E41DC00AE8C8
:1011C00015E41AC002E915E417C004E915E414C0D7
:1011D00001E216E411C003E216E40EC004E216E4D4
:1011E0000BC005E216E408C006E216E405C007E2FB
:1011F00016E402C00AE216E4C801DF91CF911F9104
:101200000F91089596E0799FF001112494E5899F4C
:10121000E00DF11D1124E60FF11DEE0FFF1FEA583E
:10122000FE4F85919491803E9105E0F4803C9105BC
:1012300058F58133910509F46FC048F4893291055E
:1012400009F463C08A32910509F46DC072C0893314
:101250009105E9F082389105D1F08533910509F4C3
:101260004DC067C0833E910581F138F4803E910501
:10127000B9F0823E9105D9F05CC0863E910561F1DE
:10128000873E9105A1F155C00E94BF0608952091A7
:10129000FA0120FD02C021FF4CC080EE90E049C061
:1012A0008091FA0180FFF9CF89E390E042C08091FC
:1012B000FA0182FF0EC08091FA0184FF03C080E032
:1012C00090E037C083EE90E034C08091FA0182FF55
:1012D000F2CF82EE90E02DC08091FA0183FF0BC027
:1012E0008091FA0184FDEBCF87EE90E022C08091DF
:1012F000FA0183FFF5CF86EE90E01BC08091FA01E2
:1013000085FF07C089E290E014C08091FA0185FF53
:10131000F9CF85E390E00DC08091FA0186FF07C008
:101320008AE290E006C08091FA0186FFF9CF81E35E
:1013300090E00E94CF06089508950C949C09809136
:101340006E010895CF93DF9300D01F92CDB7DEB723
:101350009C018091F101843019F593E099833B83DE
:101360002A839093E9008FEF9091E800815095FDDA
:1013700006C095ED9A95F1F700008111F5CF8091A7
:10138000E80085FF0DC040E050E063E070E0CE0172
:1013900001960E940C0C8091E8008E778093E80003
:1013A0000F900F900F90DF91CF910895CF93DF931F
:1013B00000D01F92CDB7DEB72091F101243021F586
:1013C00022E029839B838A8383E08093E9008FEF67
:1013D0009091E800815095FD06C095ED9A95F1F742
:1013E00000008111F5CF8091E80085FF0DC040E03D
:1013F00050E063E070E0CE0101960E940C0C8091F9
:10140000E8008E778093E8000F900F900F90DF91A7
:10141000CF9108952091F1012430F1F422E020933E
:10142000E9002FEF3091E800215035FD06C035ED81
:101430003A95F1F700002111F5CF2091E80025FF42
:101440000BC040E050E065E070E00E940C0C809121
:10145000E8008E778093E8000895CF93DF93EC0146
:101460009091F101943009F046C080910C018823DD
:10147000D9F080910D018823B9F09093E9008FEFA6
:101480009091E800815095FD06C095E19A95F1F79D
:1014900000008111F5CF8091E80085FF2CC040E06D
:1014A00050E060E170E017C081E08093E9008FEFC9
:1014B0009091E800815095FD06C095ED9A95F1F761
:1014C00000008111F5CF8091E80085FF14C040E055
:1014D00050E068E070E0CE010E940C0C8091E800C2
:1014E0008E778093E80080E1FE01AEE5B1E00190E7
:1014F0000D928A95E1F7DF91CF9108958091F001E7
:10150000811109C00E94A10D0E94FE0D8091E20090
:1015100084608093E20008951092F0010895089588
:101520000C94E5220E94461C0E94EB220E94A4100B
:101530000C949D0942E061EC81E00E941B0D42E0A9
:1015400061EC82E00E941B0D42E061EC83E00E94AE
:101550001B0D42E161EC84E00C941B0D8091F301C2
:10156000833009F455C030F4813071F0823009F4D1
:101570008EC008958A3009F47AC08B3009F460C0B7
:10158000893009F09CC020C08091F201813A09F0B5
:1015900096C08091E800877F8093E8008091F601F3
:1015A0009091F701892B21F460E18EE591E003C071
:1015B00060E080E090E070E00E94570C8091E800CD
:1015C0008B778093E80008958091F201813209F0D1
:1015D00076C08091F6019091F701009719F003977A
:1015E00009F06DC08091E800877F8093E8008091CA
:1015F000E80082FD05C08091F1018111F8CF5FC044
:101600008091F10080936E018091E8008B7753C048
:101610008091F201813A09F052C08091F6019091D7
:10162000F701892B09F04BC08091E800877F8093F8
:10163000E8008091E80080FFFCCF80910C0136C06B
:101640008091F2018132D9F58091F6019091F701F4
:10165000892BA9F58091E800877F8093E8000E949C
:10166000500D8091F40180930C010C943D158091F4
:10167000F201813221F58091E800877F8093E800B4
:101680000E94500D8091F50180936F010895809123
:10169000F201813AA1F48091E800877F8093E8000D
:1016A0008091E80080FFFCCF80916F018093F10072
:1016B0008091E8008E778093E8000C94500D089597
:1016C00084B7877F84BF88E10FB6F8948093600069
:1016D000109260000FBE90E080E80FB6F8948093FF
:1016E0006100909361000FBE0E94F3100E94A10D53
:1016F0000E94FE0D8091E20084608093E200789465
:101700000E9484100E94F51082E091E00E949F10D8
:101710000E94D3228091F101853069F40E940D1C52
:101720008091EF018823B1F30E94381C882391F344
:101730000E94F60BEFCF0E94FB10ECCF292F33272E
:1017400023303105C9F064F42130310581F02230B5
:10175000310509F043C08DE690E02AE434E042C050
:1017600021323105F1F02232310541F137C082E1F9
:1017700090E027EB34E036C099278130910541F0A5
:101780008230910541F0892B49F5E6E4F4E005C08B
:10179000EEE2F4E002C0E6E1F4E0849190E09F0123
:1017A00021C06430D8F4E62FF0E0EE0FFF1FEE5DAD
:1017B000FE4F2081318189E090E014C0643070F4E4
:1017C00070E0FB01EE0FFF1FE65EFE4F20813181CE
:1017D000FB01EA5EFE4F808190E004C080E090E073
:1017E00020E030E0FA0131832083089580E189BD53
:1017F00082E189BD09B400FEFDCF8091D8008F7DC4
:101800008093D8008091E00082608093E000809116
:10181000E00081FDFCCF0895CF92DF92EF92FF921E
:101820000F931F93CF93DF93EC018B016A010E940A
:101830006F0D811133C0C114D10439F0F6018081DC
:101840009181081B190BC80FD91FE12CF12C011530
:10185000110519F18091E80085FD16C08091E8001E
:101860008E778093E800C114D10449F0F60180819D
:101870009181E80EF91EF182E08285E00FC00E949E
:101880006F0D882321F30AC089918093F1000150E4
:101890001109FFEFEF1AFF0ADACF80E0DF91CF9155
:1018A0001F910F91FF90EF90DF90CF9008952091BE
:1018B000F8013091F9012617370748F061157105D5
:1018C00039F42091E8002E772093E80001C0B90197
:1018D00040E061157105A9F12091F101222309F47D
:1018E00043C0253009F442C02091E80023FD40C0E8
:1018F0002091E80022FD32C02091E80020FFE9CFCE
:101900004091F3002091F20030E0342BFC01CF0134
:101910006115710559F02830310540F481918093AB
:10192000F100615071092F5F3F4FF1CF41E0283046
:10193000310509F040E02091E8002E772093E8007F
:10194000C8CF4111C9CF0AC08091F101882361F04D
:10195000853061F08091E80083FD0AC08091E80045
:1019600082FFF2CF80E0089582E0089583E0089539
:1019700081E008952091F8013091F9012617370789
:1019800048F06115710539F42091E8002E77209315
:10199000E80001C0B901FC0120E06115710591F179
:1019A0008091F101882309F440C0853009F43FC0DB
:1019B0008091E80083FD3DC08091E80082FD2FC04A
:1019C0008091E80080FFE9CF2091F3008091F20040
:1019D00090E0922B6115710559F08830910540F423
:1019E00024912093F1003196615071090196F2CF54
:1019F00021E0089709F020E08091E8008E7780933D
:101A0000E800CBCF2111CCCF0AC08091F10188230F
:101A100061F0853061F08091E80083FD0AC080911B
:101A2000E80082FFF2CF80E0089582E0089583E02D
:101A3000089581E00895982F973058F59093E90024
:101A4000981739F07091EC002091ED005091F00062
:101A500003C0242F762F50E021FF19C03091EB00F6
:101A60003E7F3093EB003091ED003D7F3093ED00F1
:101A70003091EB0031603093EB007093EC002093D9
:101A8000ED005093F0002091EE0027FF07C09F5F0C
:101A9000D3CF8F708093E90081E0089580E00895AE
:101AA0008091F20187FF11C08091E80082FD05C09E
:101AB0008091F1018111F8CF11C08091E8008B77FE
:101AC0000BC08091F101882349F08091E80080FFEC
:101AD000F8CF8091E8008E778093E80008952091F8
:101AE000E4003091E50095E64091EC00842F817090
:101AF00040FF22C08091E80080FD1CC08091F10170
:101B0000882391F0853091F08091EB0085FD10C025
:101B10004091E4005091E5004217530729F39A01E0
:101B2000915011F784E0089582E0089583E00895CC
:101B300081E0089580E008954091E80042FFDECF03
:101B400008950E940F0E0E94170EE0EEF0E08081D3
:101B500081608083E8EDF0E080818F77808319BC1D
:101B6000A7EDB0E08C918E7F8C9380818F7E8083F7
:101B70001092F00108950F931F93CF93DF930E946B
:101B80000F0E0E94170EC8EDD0E088818F778883F2
:101B900088818068888388818F7D888319BC1092B2
:101BA000F1011092ED011092EF011092EE0100EEA2
:101BB00010E0F80180818B7F808388818160888339
:101BC00042E060E080E00E941B0DE1EEF0E08081E9
:101BD0008E7F8083E2EEF0E080818160808380816F
:101BE00088608083F80180818E7F80838881806116
:101BF0008883DF91CF911F910F910895E8EDF0E078
:101C000080818F7E8083E7EDF0E08081816080833A
:101C100084E082BF81E08093F0010C94BB0DE8ED7D
:101C2000F0E080818E7F80831092E2000895109210
:101C3000DA001092E10008951F920F920FB60F92F2
:101C400011242F933F934F935F936F937F938F93C1
:101C50009F93AF93BF93EF93FF938091E10082FF37
:101C60000BC08091E20082FF07C08091E1008B7F72
:101C70008093E1000E9483108091DA0080FF1FC0F2
:101C80008091D80080FF1BC08091DA008E7F809306
:101C9000DA008091D90080FF0DC080E189BD82E12A
:101CA00089BD09B400FEFDCF81E08093F1010E945F
:101CB0007E0A05C019BC1092F1010E948C0A809125
:101CC000E10080FF19C08091E20080FF15C0809183
:101CD000E2008E7F8093E2008091E2008061809339
:101CE000E2008091D80080628093D80019BC85E022
:101CF0008093F1010E94900A8091E10084FF30C03E
:101D00008091E20084FF2CC080E189BD82E189BD21
:101D100009B400FEFDCF8091D8008F7D8093D8005C
:101D20008091E1008F7E8093E1008091E2008F7EC0
:101D30008093E2008091E20081608093E2008091D4
:101D4000ED01882311F084E007C08091E30087FD56
:101D500002C081E001C083E08093F1010E94920AF9
:101D60008091E10083FF29C08091E20083FF25C0BC
:101D70008091E100877F8093E10082E08093F10110
:101D80001092ED018091E1008E7F8093E1008091BF
:101D9000E2008E7F8093E2008091E2008061809378
:101DA000E20042E060E080E00E941B0D8091F000C4
:101DB00088608093F0000E948F0AFF91EF91BF919D
:101DC000AF919F918F917F916F915F914F913F91D3
:101DD0002F910F900FBE0F901F9018951F920F928A
:101DE0000FB60F9211242F933F934F935F936F93EE
:101DF0007F938F939F93AF93BF93CF93DF93EF9393
:101E0000FF93C091E900CF708091EC00D82FD17082
:101E100080FDD0E81092E9008091F000877F8093E8
:101E2000F00078940E94320F1092E9008091F00047
:101E300088608093F000CD2BCF70C093E900FF91B4
:101E4000EF91DF91CF91BF91AF919F918F917F9152
:101E50006F915F914F913F912F910F900FBE0F9017
:101E60001F9018951F93CF93DF93CDB7DEB7AA9736
:101E70000FB6F894DEBF0FBECDBFE2EFF1E088E011
:101E80008E0F9091F10091938E13FBCF0E94AE0ABA
:101E90008091E80083FF1FC18091F2019091F301CE
:101EA000492F50E04A30510508F015C1FA01EA5AAD
:101EB000FF4F0C946D24803881F0823809F00BC1FB
:101EC0008091F6018F708093E9008091EB0085FB93
:101ED000882780F91092E90006C08091EE01909168
:101EE000EF01911182609091E800977F9093E80054
:101EF0008093F1001092F100C8C0282F2D7F09F0C7
:101F0000EAC0882319F0823061F0E5C08091F401C5
:101F1000813009F0E0C0933009F080E08093EF0158
:101F20002BC08091F401811127C08091F6018F7040
:101F300009F4D1C08093E9002091EB0020FF1CC080
:101F4000933021F48091EB00806214C09091EB00FB
:101F500090619093EB0021E030E0A90102C0440FB2
:101F6000551F8A95E2F74093EA001092EA008091AB
:101F7000EB0088608093EB001092E9008091E8000C
:101F8000877F86C08111A7C01091F4011F778091CF
:101F9000E3008078812B8093E3008091E800877FC5
:101FA0008093E8000E94500D8091E80080FFFCCFF4
:101FB0008091E30080688093E300111102C082E009
:101FC00001C083E08093F10186C08058823008F020
:101FD00082C08091F4019091F5018C3D53E095070A
:101FE00079F583E08A838AE289834FB7F894DE012A
:101FF000139620E03EE051E2E32FF0E050935700CB
:10200000E49120FF03C0E295EF703F5FEF708E2FE9
:1020100090E0EA3010F0C79601C0C0968D939D9372
:102020002F5F243149F74FBF8091E800877F80936D
:10203000E8006AE270E0CE0101960E94570C14C0DD
:10204000AE014F5F5F4F6091F6010E949E0BBC0195
:10205000009709F440C09091E800977F9093E800C2
:1020600089819A810E94BA0C8091E8008B778093D5
:10207000E80031C0803879F58091E800877F80934F
:10208000E8008091ED018093F1008091E8008E7767
:102090008093E8000E94500D1EC081111CC09091D9
:1020A000F4019230C0F48091E800877F8093E800CB
:1020B0009093ED010E94500D8091ED01811106C0B9
:1020C0008091E30087FD02C081E001C084E080933D
:1020D000F1010E949A0A8091E80083FF0AC0809172
:1020E000E800877F8093E8008091EB008062809316
:1020F000EB00AA960FB6F894DEBF0FBECDBFDF91FE
:10210000CF911F9108950895CF938091F101882375
:10211000A1F0C091E900CF709091EC00892F8170FF
:1021200090FD80E8C82B1092E9008091E80083FDC3
:102130000E94320FCF70C093E900CF910895909321
:102140007501809374010895E0917401F091750117
:10215000309721F00190F081E02D099480E00895FE
:10216000E0917401F0917501309721F00280F381C4
:10217000E02D09940895E0917401F0917501309774
:1021800021F00480F581E02D0994089520917201D9
:10219000309173018217930771F0909373018093CC
:1021A0007201E0917401F0917501309721F0068081
:1021B000F781E02D0994089520917001309171010B
:1021C0008217930771F09093710180937001E091F1
:1021D0007401F0917501309721F00084F185E02DB4
:1021E0000994089508950C94F2100E944C1C0E94CA
:1021F000BB030C940E1D9F92AF92BF92CF92DF92C1
:10220000EF92FF920F931F93CF93DF9300D000D0F4
:1022100000D0CDB7DEB70E94D3030DE010E0AA24B2
:10222000A394B12C902E802F0E94C10498012958AC
:102230003E4F6901F901F080F826A1F4015011091F
:1022400088F78FEF89838A831B820E94551C8160E7
:10225000782F9D838C8349815A816B818D810E9467
:1022600092112FC09091DA0191FF04C08E830E94D9
:10227000C7048E8125E030E0A501022E01C0440F85
:102280000A94EAF7E42E4F21C1F029839A828E2125
:1022900091E009F490E09B830E94551C8160782FA7
:1022A0009D838C8349815A816B818D810E9492111B
:1022B000F6018081E826E08204C021503109E0F671
:1022C000BDCF0E94F51F109176010E94A41018172F
:1022D000B9F00E94A4108093760126960FB6F89468
:1022E000DEBF0FBECDBFDF91CF911F910F91FF9049
:1022F000EF90DF90CF90BF90AF909F900C949D098E
:1023000026960FB6F894DEBF0FBECDBFDF91CF91FA
:102310001F910F91FF90EF90DF90CF90BF90AF9003
:102320009F900895CF93DF93CDB7DEB72B970FB66D
:10233000F894DEBF0FBECDBF4F83588769877A8779
:102340008B87DE01119686E0FD0111928A95E9F7EF
:1023500085E0FE01379601900D928A95E1F749815B
:102360005A816B817C818D819E810E94DB172B9627
:102370000FB6F894DEBF0FBECDBFDF91CF910895A9
:10238000CF93882309F4C2C0C82F823859F40E9421
:10239000A41081FDBBC089E30E94B51A0E94821B74
:1023A00089E30CC0833879F40E94A41080FDAEC08C
:1023B00083E50E94B51A0E94821B83E50E94F71AEA
:1023C000CF910C94821B843859F40E94A41082FD92
:1023D0009DC087E40E94B51A0E94821B87E4EECF5D
:1023E0008CEF8C0F813A48F48C2F0E943822811197
:1023F0008DC08C2F0E94B51AE3CF80E28C0F8830FD
:1024000048F4C77081E001C0880FCA95EAF70E94BE
:102410003B1BD6CF8BE58C0F833078F4C53A29F07F
:10242000C63A31F083E890E005C081E890E002C050
:1024300082E890E0CF910C94C61088E58C0F833130
:1024400008F064C0C83A39F1C93A41F1CA3A49F1D1
:10245000CB3A51F1CC3A59F1CD3A61F1C03B69F137
:10246000CE3A71F1CF3A79F1C13B81F1C23B89F1AA
:10247000C33B91F1C43B99F1C53BA1F1C63BA9F126
:10248000C73BB1F1C83BB9F1C93BC1F1CA3BC9F186
:1024900080E090E038C082EE90E035C089EE90E0B8
:1024A00032C08AEE90E02FC085EB90E02CC086EB26
:1024B00090E029C087EB90E026C08CEC90E023C030
:1024C0008DEC90E020C083E891E01DC08AE891E0A7
:1024D0001AC082E991E017C084E991E014C081E25A
:1024E00092E011C083E292E00EC084E292E00BC061
:1024F00085E292E008C086E292E005C087E292E0C1
:1025000002C08AE292E0CF910C94DC10CF91089542
:10251000882309F44BC0823859F40E94A41081FF2B
:1025200045C089E30E94B51A0E94821B89E30CC052
:10253000833871F40E94A41080FF38C083E50E94A4
:10254000B51A0E94821B83E50E94F71A0C94821B25
:10255000843859F40E94A41082FF28C087E40E94A6
:10256000B51A0E94821B87E4EFCF9CEF980F913A37
:1025700058F390E2980F983050F4877091E001C0C2
:10258000990F8A95EAF7892F0E94411BDFCF9BE5BF
:10259000980F933020F480E090E00C94C610885A95
:1025A000833120F480E090E00C94DC1008958823BF
:1025B00021F00E943B1B0C94821B0895882321F07C
:1025C0000E94411B0C94821B08957F928F929F92D0
:1025D000AF92BF92CF92DF92EF92FF920F931F9331
:1025E000CF93DF931F92CDB7DEB77C01C62E772E37
:1025F000FC01058102950F70128111110E94581B78
:102600000E94AE1A882379F0112369F080E28C0DC4
:10261000883048F082E00E94971A0E94AE1A91E03A
:10262000D82ED92601C0D12CE72DE295EF70F0E02D
:10263000E05AFF4F0C946D24872D807F072D0F707B
:10264000882311F00295007F112389F0002309F4FB
:1026500090C180E28C0D883020F4802F0E943B1BBB
:1026600003C0802F0E944B1B0E94821B82C18C2DB5
:102670000E948812002309F495C180E28C0D8830F5
:1026800020F4802F0E94411B03C0802F0E94511B09
:102690000E94821B87C1972D907F872D8F7090326B
:1026A00011F08295807FCC2021F0F1E0CF16B1F0BF
:1026B0001EC0112349F0002309F414C1013009F0B0
:1026C00011C10E946B1B6EC1002319F0013009F487
:1026D00069C189830E946E1B89810AC1112321F07F
:1026E000023008F05FC1FEC001115CC101C11123BD
:1026F00021F0002309F4F6C03CC1002309F4F8C01E
:102700003EC1872D86958695837090E0009719F0DD
:10271000019761F047C1112321F08C2D972D937003
:1027200002C080E090E00E94C6103CC1112321F05D
:102730008C2D972D937002C080E090E00E94DC10F9
:1027400031C18C2D112319F00E94FD1E02C00E9480
:10275000651F0E94EA1F26C1872D837009F052C0B1
:10276000111120C18C2D829586958770880F880F56
:102770009C2D9F70892E912CA12CB12C082E04C069
:10278000880C991CAA1CBB1C0A94D2F7C4FE14C066
:102790000FE010E020E030E0B901A80104C0440FD0
:1027A000551F661F771F8A95D2F7CB01BA01609536
:1027B00070958095909503C060E070E0CB01272D67
:1027C00026952695237030E02230310569F02330BC
:1027D000310589F0682979298A299B292130310519
:1027E00071F00E942319DEC0682979298A299B2962
:1027F0000E943F19D7C00E942319C501B4010E944D
:102800000719D0C0112319F0872D817001C086955A
:10281000882309F4C7C08C2D829586958770880F10
:10282000880F9C2D9F70892E912CA12CB12C082EE5
:1028300004C0880C991CAA1CBB1C0A94D2F7C4FEC5
:1028400014C00FE010E020E030E0B901A80104C09E
:10285000440F551F661F771F8A95D2F7CB01BA0127
:10286000609570958095909503C060E070E0CB0115
:10287000272D269526952370422F50E04230510592
:1028800069F04330510589F0682979298A299B2903
:102890004130510571F00E94FD1984C068297929E1
:1028A0008A299B290E94191A7DC00E94FD19C50121
:1028B000B4010E94E11976C08C2D90E0FC01E05E2D
:1028C000F109E531F10508F050C0E059FF4F0C94D3
:1028D0006D240C2D0F70872D8F71112331F00E9404
:1028E0007A19802F0E94D7125DC00E949B19802FF9
:1028F0000E94DE1257C0112339F0011153C0872DF9
:102900008F710E94C0194EC0023008F04BC0F7CF43
:10291000112339F0872D8F710E947A1943C011233A
:10292000C9F3872D8F710E949B193CC0112329F098
:10293000872D8F710E94651935C00E945B1932C0C6
:10294000112351F0172D1F71812F0E947A1963E016
:10295000812F0E948E1A26C081E00E94971A0230B1
:1029600008F182E00E94971A1DC0112331F0002364
:1029700089F28C2D0E94C01115C0002391F28C2D7C
:102980000E9488120FC0472D4F706C2DC7010E9406
:102990009D050E947F1806C0472D4F706C2DC70102
:1029A0000E94AC06DD20F9F00E948A1A80FD1BC04F
:1029B000F70112820E94841A0E947A19C7010E94AC
:1029C00002150E94841A0F90DF91CF911F910F91F1
:1029D000FF90EF90DF90CF90BF90AF909F908F903F
:1029E0007F900C949B190F90DF91CF911F910F91C5
:1029F000FF90EF90DF90CF90BF90AF909F908F901F
:102A00007F9008950F931F93CF93DF93EC018881FC
:102A100099812B813C81232BB9F09F3F11F48F3F8B
:102A200099F0CE010E940406882371F068817981B3
:102A30008A810E94801A8C010E94351A0E94FC181B
:102A4000B801CE010E94E512DF91CF911F910F9145
:102A500008950E94581B0E94681B0E942D1B0E9413
:102A6000821B0E949B200E94EA1F80E090E00E944F
:102A7000C61080E090E00C94DC100E94481B0C947F
:102A800029150E94751A292F22952F7030E02C30BD
:102A900031054CF42A3031056CF4225031092230D2
:102AA0003105A8F407C02C30310569F02F3031050D
:102AB00051F00DC0803F69F018F4803E40F409C029
:102AC000843F29F406C093FB882780F9089580E0AD
:102AD000089581E00895CF93DF9300D000D01F9236
:102AE000CDB7DEB70F900F900F900F900F90DF9142
:102AF000CF910895CF93DF9300D000D000D0CDB711
:102B0000DEB726960FB6F894DEBF0FBECDBFDF91BD
:102B1000CF9108951F93CF93DF93C091850116E065
:102B200080918601C81799F0D0E01C9FF0011D9F8D
:102B3000F00D1124E957FE4F40815181628173816C
:102B4000848195810E947A152196C770E9CFDF9123
:102B5000CF911F9108954091B7015091B8016091B4
:102B6000B9017091BA018091BB019091BC010C94A4
:102B70007A158091BC0182958F7009F054C08091C4
:102B8000B901882309F44FC080918501A091860185
:102B90006091B7017091B8014091BA015091BB01A9
:102BA000B6E08A1709F43FC090E041155105C1F124
:102BB0007F3F11F46F3FA1F1B89FF001B99FF00D75
:102BC0001124E957FE4F218172132AC0208162131C
:102BD00027C02281211124C0238134812417350785
:102BE00010F421503109241B350B283C3105C0F469
:102BF0002091BC012F7020612093BC0126E0289F0A
:102C0000F001299FF00D1124E457FE4F80818F7051
:102C10008061808387EB91E00E9402150C948A15F5
:102C200001968770BECF0895CF92DF92EF92FF9208
:102C30000F931F93CF93DF93CDB7DEB762970FB695
:102C4000F894DEBF0FBECDBF8C0185E0F801DE0138
:102C50001D9601900D928A95E1F7D8014C9111963D
:102C60005C91119712966C9112971396CD90DC900F
:102C700014973091B7017091B8018091BA01909189
:102C8000BB01009709F46BC17F3F19F43F3F09F482
:102C900066C1E090B901EE2009F4C0C02091BC01EA
:102CA000C816D90628F0F601E81BF90BCF0104C0BD
:102CB000809590958C0D9D1DFF24F394883C910583
:102CC00078F0F12C207F09F0C6C07C2DD98AC88A03
:102CD00089890E946B1587EB91E00E940215B1C0B3
:102CE000822F807F09F046C0751314C0341312C0C0
:102CF000611110C02F7020612093BC010E94AB15A0
:102D000087EB91E00E9402158091BC01D8011596D5
:102D10008C932EC0CD2819F15F3F11F44F3FF9F08D
:102D2000F62E61111CC0809185012091860136E04C
:102D3000821709F45AC090E0389FF001399FF00DD6
:102D40001124E957FE4F7181571306C07081471354
:102D500003C07281711103C001968770E9CFF62E0E
:102D6000662309F418C18091BC0181608093BC0185
:102D7000F12C11C1751308C0341306C0611104C0D1
:102D80008091BC01D801C3C04D875E878D859E852B
:102D90006A8B0E9441156A898823E1F16623D1F18B
:102DA0002091BC01822F82958F7090E0029774F081
:102DB0008091B7019091B80198878F831986DB863F
:102DC000CA862C87CE0107960E94021586E0F8017C
:102DD000A7EBB1E001900D928A95E1F70E94B91539
:102DE0000E94AB15FF24F394D6C04D875E878D8576
:102DF0009E850E94751A292F22952F7030E022306F
:102E000031050CF0BCC09F7009F0B6C0805E883000
:102E100008F4C1C0C8010E940215E4CFC816D90643
:102E200008F453C0F601E81BF90BCF01883C91056B
:102E300008F450C0F12C7C2DD98AC88A89890E9457
:102E40006B15E7EBF1E086E0DF011D928A95E9F76B
:102E50000E94AB15A0C0751314C0341312C06111C9
:102E600010C08091BC01F8018583C8010E94021541
:102E700086E0E7EBF1E0DF011D928A95E9F7FE2C91
:102E80008AC04D875E878D859E856A8B0E9441151D
:102E90006A89882309F4BECF662309F4BBCF209149
:102EA000BC01822F82958F7090E002970CF48ECF38
:102EB0008091B7019091B8019A8389831B82DD824A
:102EC000CC822E83CE0101967FCF809590958C0D7C
:102ED0009D1DACCFF62E662309F49CCF75132EC032
:102EE00034132CC02091BC0120FD1FC0822F82957D
:102EF0008F70D9F0D80115962C9315978F3049F023
:102F00008F5F982F9295907F822F8F70892B1596C7
:102F10008C93C8010E94021586E0F801A7EBB1E08E
:102F200001900D928A95E1F793CF86E0F801A7EB27
:102F3000B1E001900D928A95E1F72DC04D875E8733
:102F40008D859E850E944115811140CF8091BC01E5
:102F500081608093BC01C8010E9402151CC06623D9
:102F600009F458CF4D875E878D859E850E94411557
:102F7000882309F44FCF2ACF811148CF0CC02430C9
:102F800031050CF047CF9F7009F440CFF8019581CF
:102F9000907F09F03BCF8F2D62960FB6F894DEBF7D
:102FA0000FBECDBFDF91CF911F910F91FF90EF909A
:102FB000DF90CF9008951F93CF93DF93CDB7DEB707
:102FC0002C970FB6F894DEBF0FBECDBF4F83588746
:102FD00069877A878B879C87CE0107960E94141693
:102FE000882369F08F8198852A853B85232BF1F111
:102FF0009F3F09F063C08F3F09F060C037C086E093
:10300000FE013796DE01119601900D928A95E1F747
:103010006F817885EA85FB85309741F17F3F11F418
:103020006F3F21F12091860130E0C9010196877040
:1030300099274091850150E08417950709F447C00E
:1030400069837A83FD83EC8396E0929FD001939FFE
:10305000B00D1124A957BE4FFE01319601900D927B
:103060009A95E1F7809386010E948A1516E0809177
:103070008501909186018917C1F1189FC001112423
:1030800089579E4F0E941416882379F1E09185019B
:103090001E9FF0011124E957FE4F4081518162814A
:1030A0007381848195810E947A158091850190E0D9
:1030B00001968770992780938501D9CF4F815885D4
:1030C00069857A858B859C850E947A15CFCF0E9471
:1030D0003D151092860110928501E7EBF1E086E044
:1030E000DF011D928A95E9F7C1CF2C960FB6F894AF
:1030F000DEBF0FBECDBFDF91CF911F910895EF923C
:10310000FF920F931F93CF93DF938C01009709F4E5
:103110006CC0F12CEE24E394E8012196F80184912F
:10312000843740F4843008F051C0813081F082301F
:1031300019F15BC0853709F444C0A8F19CE7980FEA
:10314000903708F052C08F770E94881241C00E5FFE
:103150001F4FFE01C49180E28C0F883048F4C77085
:103160008E2D01C0880FCA95EAF70E945B1B14C020
:103170008C2F0E94C0112DC00E5F1F4FFE01C49105
:1031800080E28C0F883058F4C7708E2D01C0880FF4
:10319000CA95EAF70E94611B0E94821B1AC08C2FFD
:1031A0000E94881216C00E5F1F4FFE01C491CC23EF
:1031B00081F08FE99FE00197F1F700C00000C15056
:1031C000F6CF0E5F1F4FFE01F49003C00E94C011A6
:1031D0008E018F2D882309F49FCFEFE9FFE031970F
:1031E000F1F700C000008150F5CFDF91CF911F9122
:1031F0000F91FF90EF90089508956093C10170932F
:10320000C2018093C3019093C4010C9429150F93BC
:103210001F930091C1011091C2012091C30130910F
:10322000C401DC01CB01802B912BA22BB32B80930B
:10323000C1019093C201A093C301B093C4011F9137
:103240000F910C9429150F931F930091C1011091B8
:10325000C2012091C3013091C401DC01CB01802364
:103260009123A223B3238093C1019093C201A09321
:10327000C301B093C4011F910F910C9429150F93B2
:103280001F930091C1011091C2012091C30130919F
:10329000C401DC01CB0180279127A227B3278093AB
:1032A000C1019093C201A093C301B093C4011F91C7
:1032B0000F910C9429151092BD011092BE0110922D
:1032C000BF011092C0010C94291541E050E060E06C
:1032D00070E004C0440F551F661F771F8A95D2F710
:1032E0004093BD015093BE016093BF017093C00134
:1032F0000C94291541E050E060E070E004C0440FF8
:10330000551F661F771F8A95D2F78091BD01909156
:10331000BE01A091BF01B091C001482B592B6A2B6F
:103320007B2B4093BD015093BE016093BF0170930E
:10333000C0010C94291541E050E060E070E004C049
:10334000440F551F661F771F8A95D2F740955095F9
:10335000609570958091BD019091BE01A091BF01D3
:10336000B091C001482359236A237B234093BD01B8
:103370005093BE016093BF017093C0010C94291556
:1033800041E050E060E070E004C0440F551F661F4C
:10339000771F8A95D2F78091BD019091BE01A091CF
:1033A000BF01B091C001482759276A277B27409366
:1033B000BD015093BE016093BF017093C0010C9496
:1033C00029150F931F930091BD011091BE0120910B
:1033D000BF013091C001DC01CB01802B912BA22BCE
:1033E000B32B8093BD019093BE01A093BF01B09316
:1033F000C0011F910F910C9429150F931F930091F9
:10340000BD011091BE012091BF013091C001DC01CE
:10341000CB0180239123A223B3238093BD019093FA
:10342000BE01A093BF01B093C0011F910F910C94F6
:1034300029150F931F930091BD011091BE0120919A
:10344000BF013091C001DC01CB0180279127A22769
:10345000B3278093BD019093BE01A093BF01B093A9
:10346000C0011F910F910C9429150895CF92DF92FE
:10347000EF92FF920F931F93CF93DF938C01C09035
:10348000C101D090C201E090C301F090C4018091CD
:10349000BD019091BE01A091BF01B091C001C82AA9
:1034A000D92AEA2AFB2ACFE1D0E0D701C6010C2EA7
:1034B00004C0B695A795979587950A94D2F780FF93
:1034C00006C0B8018C2F0E940209019721F42197B0
:1034D00060F780E001C08C2FDF91CF911F910F9199
:1034E000FF90EF90DF90CF900895CF93DF93EC01A2
:1034F0000E94361ABE010E940209DF91CF91089501
:10350000CB010E94751A08958091C5018595859516
:10351000859508958091C5018770089598E0899FE9
:1035200090011124262B2093C5010C947A19209127
:10353000C501809582238093C501982F977069F407
:1035400030E0482F552747FD50952417350729F0BF
:103550008595859585950C949B1908959091C50145
:10356000977081E009F480E0089590910C0199230F
:1035700021F090910D01911109C020910E0130911F
:103580000F01F90132969FEF40E01FC0982F9695EA
:10359000969596959F3050F5E0910E01F0910F01B0
:1035A000E90FF11D877021E030E0A90102C0440F4E
:1035B000551F8A95E2F7CA019181892B818308956D
:1035C0009F3F39F04F5F4E3041F051915813F8CF83
:1035D0000DC05111F7CF942FF5CF9F3F39F0F9016E
:1035E000E90FF11D97FDFA95828308950895909152
:1035F0000C01992321F090910D01911109C02091A6
:103600000E0130910F01F9013296205F3F4F1FC02C
:10361000982F9695969596959F30F0F4E0910E012F
:10362000F0910F01E90FF11D877021E030E0A90151
:1036300002C0440F551F8A95E2F7CA018095918117
:103640008923818308953196E217F30729F0908149
:103650009813F9CF1082F7CF089581E090E0E091C0
:103660000E01F0910F01E80FF91F108201968031D1
:103670009105A9F708959091D901892B8093D901DB
:10368000089580959091D90189238093D901089557
:103690001092D90108959091D801892B8093D80177
:1036A000089580959091D80189238093D801089539
:1036B0001092D80108959091D701892B8093D7015A
:1036C000089580959091D70189238093D70108951B
:1036D0001092D70108958093C60108951092C601F3
:1036E000089580910E0190910F01FC0131969C018B
:1036F000205F3F4F80E0919191118F5FE217F307B8
:10370000D1F70895E0910E01F0910F018091D90158
:103710008083E0910E01F0910F0190818091D8019A
:10372000892B8083E0910E01F0910F0190818091AF
:10373000D701892B80838091C601882361F0E091B5
:103740000E01F0910F019081892B80830E94711BE3
:1037500081111092C60180910E0190910F010C947D
:10376000B01020E0009739F0AC014150510984239A
:1037700095232F5FF7CF822F0895CF92DF92EF929C
:10378000FF926C01EE24FF24C114D104E104F10482
:1037900021F0C701B60120E101C020E0C72ED82EDC
:1037A000E92EFF24C114D104E104F10419F0285FCB
:1037B000C701B6016B017C0154E0F694E794D794FD
:1037C000C7945A95D1F7C114D104E104F10419F05A
:1037D0002C5FC701B6016B017C0142E0F694E794CF
:1037E000D794C7944A95D1F7C114D104E104F104E8
:1037F00019F02E5FC701B601DC01CB01B695A79584
:1038000097958795892B8A2B8B2B09F02F5F822F19
:10381000FF90EF90DF90CF9008958091F101843078
:1038200021F11092DB0120E488E190E00FB6F894DA
:10383000A895809360000FBE2093600080E00E94F6
:103840009D0983B7817F846083BF83B7816083BF15
:103850007894889583B78E7F83BF88E10FB6F894FC
:1038600080936000109260000FBE0895089508953F
:103870000E94361C0E94D3030E94371C0E94C80479
:1038800091E0811101C090E0892F08950E943D15BB
:103890000E94A4100C949D0982E084BD93E095BD24
:1038A0009AEF97BD80936E0008952FB7F89480919A
:1038B000DC019091DD01A091DE01B091DF012FBF0D
:1038C0000895CF92DF92EF92FF920F931F932FB73D
:1038D000F8944091DC015091DD016091DE0170911E
:1038E000DF012FBF6A017B01EE24FF248C0120E061
:1038F00030E0C016D106E206F30610F4415051093B
:103900009A01281B390BC9011F910F91FF90EF906D
:10391000DF90CF9008951F920F920FB60F9211244F
:103920008F939F93AF93BF938091DC019091DD01C2
:10393000A091DE01B091DF010196A11DB11D809320
:10394000DC019093DD01A093DE01B093DF01BF9114
:10395000AF919F918F910F900FBE0F901F90189570
:103960000E94A10DF8942FEF87EA91E62150804044
:103970009040E1F700C0000087E090EBDC0180930D
:10398000FB019093FC01A093FD01B093FE019CE02C
:1039900088E10FB6F894A895809360000FBE9093CD
:1039A0006000FFCFEF92FF920F931F93CF93DF93AF
:1039B000D82FCDE08C2F0E94C10405E010E0E82E46
:1039C000F12CC701002E02C0959587950A94E2F765
:1039D00080FF09C0602F7C2F80E00E94AD06D813C5
:1039E00002C081E006C00150110958F7C15010F71C
:1039F00080E0DF91CF911F910F91FF90EF9008959C
:103A0000CF93C82F8CE20E94D21C882321F08C2FE8
:103A1000CF910C94D21C80E0CF910895CF930E9457
:103A2000551E811102C00E943B1EC5E6C15049F0DF
:103A30000E94D3038FE39CE90197F1F700C00000D7
:103A4000F5CF89E20E94001D811113C18AE20E9414
:103A5000001D81110E943B1E85E00E94001D811106
:103A60000E94B01C0E94601E8093DA0187E00E94D1
:103A7000001D8823A9F18BE10E94001D882351F0CD
:103A80008091DA0181FB222720F991E0922790FBB7
:103A900081F90EC08EE00E94001D882361F08091A4
:103AA000DA0182FB222720F991E0922790FB82F92C
:103AB0008093DA0115C080E10E94001D9091DA0127
:103AC000882341F093FB222720F981E0822780FBA5
:103AD00093F904C0892F809580FB90F99093DA01C7
:103AE0008091DA010E94641E0E94721E8093FA0186
:103AF00080EE0E94001D882341F08091FA01982FEA
:103B0000909590FB80F98093FA0189E30E94001D53
:103B1000882359F08091FA0181FB222720F991E056
:103B2000922790FB81F98093FA0182EE0E94001D9A
:103B3000882359F08091FA0182FB222720F991E035
:103B4000922790FB82F98093FA0186EE0E94001D75
:103B5000882359F08091FA0183FB222720F991E014
:103B6000922790FB83F98093FA0183EE0E94001D57
:103B7000882359F08091FA0184FB222720F991E0F3
:103B8000922790FB84F98093FA0185E30E94001D3F
:103B9000882359F08091FA0185FB222720F991E0D2
:103BA000922790FB85F98093FA0181E30E94001D22
:103BB000882359F08091FA0186FB222720F991E0B1
:103BC000922790FB86F98093FA0181E10E94001D03
:103BD000882359F08091FA0187FB222720F991E090
:103BE000922790FB87F98093FA018091FA010E9455
:103BF000761E8091FA0187FB882780F980930D015A
:103C000087E20E94001DC82F8EE10E94001D8111D5
:103C1000C2608FE10E94001D8111C46080E20E9499
:103C2000001D8111C86081E20E94001D8111C061E8
:103C300082E20E94001D8111C06283E20E94001D89
:103C40008111C06484E20E94001D882311F0C068C5
:103C500002C0CC2329F08C2F0E946D1E6C2F03C054
:103C60000E94691E682F70E080E090E0CF910C9474
:103C7000FD18CF9108956DEE7EEF80E090E00E94F8
:103C8000A72460E082E090E00E94952460E083E059
:103C900090E00E94952460E084E090E00E949524EA
:103CA00060E085E090E00C94952480E090E00E9434
:103CB0008F2421E08D3E9E4F09F020E0822F089551
:103CC00082E090E00C948724682F82E090E00C94CE
:103CD000952483E090E00C948724682F83E090E0A3
:103CE0000C94952484E090E00C948724682F84E061
:103CF00090E00C9495248091E20180FF0BC06091CC
:103D0000130185E0689FB00111247595679575953D
:103D100067952BC081FF09C06091130185E0689F02
:103D2000B00111247595679520C082FF07C060918E
:103D3000130185E0689FB001112417C09091E30141
:103D40009923D1F060911201961788F72091130101
:103D500085E0289F90011124929FA001939F500D10
:103D6000112470E0CA010E9459246038710540F4A2
:103D70006115710539F002C065E070E0862F089585
:103D80008FE7089581E008958091E20180FF08C0E7
:103D90006091110170E0759567957595679521C0E3
:103DA00081FF06C06091110170E07595679519C09B
:103DB00082FF04C06091110170E010C09091E30196
:103DC0009923C1F0609110019617A0F7809111011D
:103DD000899FC001112470E00E9459246038710548
:103DE00028F46115710521F0862F08958FE7089555
:103DF00081E0089561E070E0F4CF803F21F40E94FB
:103E00007B1E819504C0813F29F40E947B1E809314
:103E1000E6010895823F21F40E947B1E819504C033
:103E2000833F29F40E947B1E8093E5010895893F1A
:103E300019F40E94C41E05C08A3F31F40E94C41EBA
:103E400081958093E70108958B3F21F40E94C41E61
:103E5000819504C08C3F29F40E94C41E8093E80120
:103E60000895843F21F48091E401816017C0853F6B
:103E700021F48091E401826011C0863F21F4809199
:103E8000E40184600BC0873F21F48091E4018860E5
:103E900005C0883F31F48091E40180618093E401A2
:103EA00008958D3F21F48091E20181600BC08E3F27
:103EB00021F48091E201826005C08F3F29F4809156
:103EC000E20184608093E2010895803F39F480919B
:103ED000E60187FF6CC01092E60169C0813F29F4BA
:103EE0008091E6011816BCF362C09091E501823F13
:103EF00029F497FF5CC01092E50159C0833F19F483
:103F00001916CCF354C0893F41F48091E70118168B
:103F10000CF04DC01092E7014AC08A3F29F480910D
:103F2000E70187FF44C0F6CF8B3F39F48091E80169
:103F300087FF3DC01092E8013AC08C3F29F4809180
:103F4000E8011816BCF333C0843F21F48091E401EA
:103F50008E7F17C0853F21F48091E4018D7F11C0D1
:103F6000863F21F48091E4018B7F0BC0873F21F4D1
:103F70008091E401877F05C0883F31F48091E4019E
:103F80008F7E8093E40113C08D3F21F48091E20184
:103F90008E7F0BC08E3F21F48091E2018D7F05C0A2
:103FA0008F3F29F48091E2018B7F8093E201809121
:103FB000E50181110EC08091E60181110AC0809156
:103FC000E701811106C08091E801811102C01092C1
:103FD000E301089584EE91E00E94BB100E94551CFD
:103FE0009093E1018093E00108951F93CF93DF93B5
:103FF0008091E0019091E1010E94611CAC019091DF
:10400000E301992321F02091140130E006C02091B2
:1040100015018AE0289F900111244217530708F4E4
:1040200086C08091E501C091E601D091E701109131
:10403000E801811107C0C11176C0D11174C01111FE
:1040400072C075C09F3F19F09F5F9093E3011816EF
:1040500024F40E947B1E8093E5018091E50187FF97
:1040600005C00E947B1E81958093E5011C1624F4F7
:104070000E947B1E8093E6018091E60187FF05C0C8
:104080000E947B1E81958093E6016091E501662385
:1040900039F1C091E601CC2319F1772767FD7095BE
:1040A000872F972F0E946A2323E333E343E35FE3E1
:1040B0000E94CE230E9437236093E5016C2F77275F
:1040C00067FD7095872F972F0E946A2323E333E3C0
:1040D00043E35FE30E94CE230E9437236093E6010F
:1040E0001D1624F40E94C41E8093E7018091E7010D
:1040F00087FF05C00E94C41E81958093E7011116B9
:1041000024F40E94C41E8093E8018091E80187FF97
:1041100005C00E94C41E81958093E801DF91CF9174
:104120001F910C94EA1F9F3F09F08ECF96CFDF912D
:10413000CF911F910895E4EEF1E085E0DF011D923B
:104140008A95E9F71092E3011092E2010895833015
:1041500081F128F4813059F08230D1F00895853012
:1041600009F449C0B8F1863009F456C00895809129
:104170001501262F30E0280F311D2F3F310524F483
:10418000680F6093150108958FEF809315010895CE
:1041900080911401262F30E0280F311D2F3F31056B
:1041A00024F4680F6093140108958FEF8093140135
:1041B000089580911301262F30E0280F311D2F3FE5
:1041C000310524F4680F6093130108958FEF8093F5
:1041D0001301089580911201262F30E0280F311D20
:1041E0002F3F310524F4680F6093120108958FEF7B
:1041F00080931201089580911101262F30E0280F3D
:10420000311D2F3F310524F4680F6093110108958B
:104210008FEF80931101089580911001262F30E0D7
:10422000280F311D2F3F310524F4680F60931001D2
:1042300008958FEF809310010895833011F128F4D1
:10424000813049F0823091F00895853081F120F17C
:104250008630C1F1089580911501681720F4861BFE
:10426000809315010895109215010895809114010D
:10427000681720F4861B809314010895109214018E
:10428000089580911301681720F4861B8093130111
:10429000089510921301089580911201681720F477
:1042A000861B809312010895109212010895809147
:1042B0001101681720F4861B809311010895109254
:1042C0001101089580911001681720F4861B8093D6
:1042D000100108951092100108950F931F938D31CE
:1042E00009F46BC008F03FC08E3009F47FC0C0F401
:1042F000873009F469C068F4863009F0B1C0809154
:10430000DA01817F8E7F8093DA0181E08093EA0178
:10431000A8C0883009F4A2C08B3009F49FC0A0C0A7
:10432000863109F49BC078F4803109F472C0813180
:1043300009F096C00E943D1590910D0181E08927FA
:1043400080930D018BC0893109F488C08B3109F04D
:1043500087C08091DA0181FB222720F991E0922722
:1043600090FB81F94CC0853309F470C048F4873262
:1043700009F46CC008F459C0893209F467C070C0F0
:10438000833438F48A3308F04EC0883309F466C0A9
:1043900067C0833409F45AC0883409F061C00E94B0
:1043A0003D150FEF13ED20E3015010402040E1F7E1
:1043B00000C000000E94B01C51C00E94F1220E9467
:1043C000A4100E949D094AC09091DA01892F80951E
:1043D000817080FB90F929F0966098609093DA01E3
:1043E00040C0997F977F9093DA0138C08091DA01BD
:1043F00082FB222720F991E0922790FB82F980939B
:10440000DA01992359F18091DA0181608093DA0110
:1044100025C08091DA0183FB222720F991E09227C1
:1044200090FB83F9ECCF895301C08D5141E050E0FE
:1044300060E070E08A019B0104C0000F111F221F81
:10444000331F8A95D2F7C901B80104C061E070E05A
:1044500080E090E00E94FD180E943D1581E001C0BF
:1044600080E01F910F91089580E0089580E0089505
:10447000CF93C82F8091EA01813079F018F0823013
:10448000E9F187C0E0910E01F0910F018081813147
:1044900069F0823209F07FC009C0E0910E01F0910D
:1044A0000F018081813111F0823261F48C2F0E94E2
:1044B0003422811104C08C2F0E946D211DC081E027
:1044C00090E01AC08C2F0E943622811114C0C43192
:1044D00079F048F4CB3079F0C03109F060C082E067
:1044E0008093EA0108C0C93219F0C83321F057C0DF
:1044F0001092EA0154C081E0817053C0C93289F141
:1045000018F5C43171F1A8F4C73009F046C08AE04B
:104510008093150194E19093140193E0909313011B
:104520008093120188E08093110188E2809310014A
:1045300034C0CE51C63088F5EC2FF0E0E65DFE4F7A
:1045400080818093E90129C0CE34E9F020F4CB3496
:1045500021F56AE013C0C13579F0C235F1F461E0AC
:104560000DC08091E901882319F01092E90115C06E
:1045700081E08093EA0115C061E006C08091E90105
:104580000E94A7200AC06AE08091E9010E941D21D3
:1045900004C01092EA0180E004C081E002C080E023
:1045A000ABCFCF910895E1E8F0E08081886080830F
:1045B0008081816080838FB7F89493E09093890025
:1045C00090ED909388008FBF0895EFE6F0E0808132
:1045D000826080830895EFE6F0E080818D7F8083A4
:1045E0000895EFE6F0E0908182E0892780830895C6
:1045F0001F920F920FB60F9211242F933F934F9358
:104600005F936F937F938F939F93AF93BF93EF933A
:10461000FF938091EB019091EC0101969093EC0156
:104620008093EB01811103C082E00E949D09E0911B
:10463000EC01E695E695F0E0EC53FA4FE4918091B9
:10464000EB018E1303C080E00E949D09FF91EF9162
:10465000BF91AF919F918F917F916F915F914F919A
:104660003F912F910F900FBE0F901F90189504D07F
:104670006894B1118DC0089570D088F09F5790F064
:10468000B92F9927B751A0F0D1F0660F771F881F77
:10469000991F1AF0BA95C9F712C0B13081F077D0DE
:1046A000B1E0089574C0672F782F8827B85F39F07C
:1046B000B93FCCF3869577956795B395D9F73EF4D6
:1046C00090958095709561957F4F8F4F9F4F08957E
:1046D000E89409C097FB3EF490958095709561959C
:1046E0007F4F8F4F9F4F9923A9F0F92F96E9BB2752
:1046F0009395F695879577956795B795F111F8CFCE
:10470000FAF4BB0F11F460FF1BC06F5F7F4F8F4F38
:104710009F4F16C0882311F096E911C0772321F02E
:104720009EE8872F762F05C0662371F096E8862FC6
:1047300070E060E02AF09A95660F771F881FDAF71D
:10474000880F9695879597F9089557FD9058440FCF
:10475000551F59F05F3F71F04795880F97FB991FE0
:1047600061F09F3F79F0879508951216130614069D
:10477000551FF2CF4695F1DF08C01616170618062A
:10478000991FF1CF86957105610508940895E89405
:10479000BB2766277727CB0197F908950BD078C000
:1047A00069D028F06ED018F0952309F05AC05FC088
:1047B0001124EECFCADFA0F3959FD1F3950F50E0FF
:1047C000551F629FF001729FBB27F00DB11D639FC3
:1047D000AA27F00DB11DAA1F649F6627B00DA11D69
:1047E000661F829F2227B00DA11D621F739FB00D0F
:1047F000A11D621F839FA00D611D221F749F33277F
:10480000A00D611D231F849F600D211D822F762F17
:104810006A2F11249F5750408AF0E1F088234AF014
:10482000EE0FFF1FBB1F661F771F881F9150504060
:10483000A9F79E3F510570F014C0AACF5F3FECF37B
:10484000983EDCF3869577956795B795F795E7954C
:104850009F5FC1F7FE2B880F911D9695879597F95D
:10486000089597F99F6780E870E060E008959FEFF2
:1048700080EC089500240A941616170618060906F7
:10488000089500240A9412161306140605060895C6
:10489000092E0394000C11F4882352F0BB0F40F44E
:1048A000BF2B11F460FF04C06F5F7F4F8F4F9F4F8E
:1048B000089597FB072E16F4009407D077FD09D0D2
:1048C0000E94732407FC05D03EF4909581959F4F7C
:1048D0000895709561957F4F0895EE0FFF1F059025
:1048E000F491E02D0994AA1BBB1B51E107C0AA1F3C
:1048F000BB1FA617B70710F0A61BB70B881F991F81
:104900005A95A9F780959095BC01CD010895F99924
:10491000FECF92BD81BDF89A992780B50895A8E190
:10492000B0E042E050E00C94AF24262FF999FECF7E
:1049300092BD81BDF89A019700B4021639F01FBAF2
:1049400020BD0FB6F894FA9AF99A0FBE0895019611
:10495000272F0E9496240C949524DC01CB01FC01A6
:10496000F999FECF06C0F2BDE1BDF89A319600B4C8
:0E4970000D9241505040B8F70895F894FFCFD3
:10497E0002209F092D0A0A0AD609A2090101C701C0
:10498E0028080A03140A3F4D3639850538050205F5
:10499E00C9045C0475048E04A70401020304050611
:0449AE0007080900ED
:00000001FF
